BL51 BANKED LINKER/LOCATER V5.03                                                        07/03/2006  11:00:03  PAGE 1


BL51 BANKED LINKER/LOCATER V5.03, INVOKED BY:
C:\KEIL\C51\BIN\BL51.EXE STARTUP.obj, SHTxx_dummy_code.obj TO SHTxx_Demo1 RAMSIZE (256) CODE (0X0000-0X1FFF)


MEMORY MODEL: SMALL


INPUT MODULES INCLUDED:
  STARTUP.obj (?C_STARTUP)
  SHTxx_dummy_code.obj (SHTXX_DUMMY_CODE)
  C:\KEIL\C51\LIB\C51S.LIB (?C?UIDIV)
  C:\KEIL\C51\LIB\C51S.LIB (?C?SIDIV)
  C:\KEIL\C51\LIB\C51S.LIB (?C?ILDPTR)
  C:\KEIL\C51\LIB\C51S.LIB (?C?ISTPTR)
  C:\KEIL\C51\LIB\C51S.LIB (?C?LMUL)
  C:\KEIL\C51\LIB\C51S.LIB (?C?ULSHR)
  C:\KEIL\C51\LIB\C51S.LIB (PRINTF)
  C:\KEIL\C51\LIB\C51S.LIB (ABS)
  C:\KEIL\C51\LIB\C51S.LIB (?C?CLDPTR)
  C:\KEIL\C51\LIB\C51S.LIB (?C?CLDOPTR)
  C:\KEIL\C51\LIB\C51S.LIB (?C?CSTPTR)
  C:\KEIL\C51\LIB\C51S.LIB (?C?PLDIIDATA)
  C:\KEIL\C51\LIB\C51S.LIB (?C?CCASE)
  C:\KEIL\C51\LIB\C51S.LIB (PUTCHAR)


LINK MAP OF MODULE:  SHTxx_Demo1 (?C_STARTUP)


            TYPE    BASE      LENGTH    RELOCATION   SEGMENT NAME
            -----------------------------------------------------

            * * * * * * *   D A T A   M E M O R Y   * * * * * * *
            REG     0000H     0008H     ABSOLUTE     "REG BANK 0"
                    0008H     0018H                  *** GAP ***
            BIT     0020H.0   0001H.1   UNIT         _BIT_GROUP_
                    0021H.1   0000H.7                *** GAP ***
            DATA    0022H     001AH     UNIT         _DATA_GROUP_
            IDATA   003CH     0001H     UNIT         ?STACK

            * * * * * * *   C O D E   M E M O R Y   * * * * * * *
            CODE    0000H     0003H     ABSOLUTE     
                    0003H     07FDH                  *** GAP ***
            CODE    0800H     035CH     UNIT         ?PR?PRINTF?PRINTF
            CODE    0B5CH     01C5H     UNIT         ?C?LIB_CODE
            CODE    0D21H     00CEH     UNIT         ?PR?_CALC_SHT10?SHTXX_DUMMY_CODE
            CODE    0DEFH     00C2H     UNIT         ?PR?MAIN?SHTXX_DUMMY_CODE
            CODE    0EB1H     0041H     UNIT         ?CO?SHTXX_DUMMY_CODE
            CODE    0EF2H     0027H     UNIT         ?PR?PUTCHAR?PUTCHAR
            CODE    0F19H     0012H     UNIT         ?PR?_ABS?ABS
            CODE    0F2BH     000DH     UNIT         ?PR?INIT_UART?SHTXX_DUMMY_CODE
            CODE    0F38H     000CH     UNIT         ?C_C51STARTUP



OVERLAY MAP OF MODULE:   SHTxx_Demo1 (?C_STARTUP)


BL51 BANKED LINKER/LOCATER V5.03                                                      07/03/2006  11:00:03  PAGE 2


SEGMENT                                     BIT_GROUP          DATA_GROUP 
  +--> CALLED SEGMENT                    START    LENGTH     START    LENGTH
----------------------------------------------------------------------------
?C_C51STARTUP                            -----    -----      -----    -----
  +--> ?PR?MAIN?SHTXX_DUMMY_CODE

?PR?MAIN?SHTXX_DUMMY_CODE                -----    -----      0022H    0006H
  +--> ?PR?INIT_UART?SHTXX_DUMMY_CODE
  +--> ?PR?_CALC_SHT10?SHTXX_DUMMY_CODE
  +--> ?CO?SHTXX_DUMMY_CODE
  +--> ?PR?PRINTF?PRINTF
  +--> ?PR?_ABS?ABS

?PR?_CALC_SHT10?SHTXX_DUMMY_CODE         -----    -----      0028H    000CH

?PR?PRINTF?PRINTF                        0020H.0  0001H.1    0028H    0014H
  +--> ?PR?PUTCHAR?PUTCHAR



SYMBOL TABLE OF MODULE:  SHTxx_Demo1 (?C_STARTUP)

  VALUE           TYPE          NAME
  ----------------------------------

  -------         MODULE        ?C_STARTUP
  C:0F38H         SEGMENT       ?C_C51STARTUP
  I:003CH         SEGMENT       ?STACK
  C:0000H         PUBLIC        ?C_STARTUP
  D:00E0H         SYMBOL        ACC
  D:00F0H         SYMBOL        B
  D:0083H         SYMBOL        DPH
  D:0082H         SYMBOL        DPL
  N:0000H         SYMBOL        IBPSTACK
  N:0100H         SYMBOL        IBPSTACKTOP
  N:0080H         SYMBOL        IDATALEN
  C:0F3BH         SYMBOL        IDATALOOP
  N:0000H         SYMBOL        PBPSTACK
  N:0000H         SYMBOL        PBPSTACKTOP
  N:0000H         SYMBOL        PDATALEN
  N:0000H         SYMBOL        PDATASTART
  N:0000H         SYMBOL        PPAGE
  N:0000H         SYMBOL        PPAGEENABLE
  D:00A0H         SYMBOL        PPAGE_SFR
  D:0081H         SYMBOL        SP
  C:0F38H         SYMBOL        STARTUP1
  N:0000H         SYMBOL        XBPSTACK
  N:0000H         SYMBOL        XBPSTACKTOP
  N:0000H         SYMBOL        XDATALEN
  N:0000H         SYMBOL        XDATASTART
  C:0000H         LINE#         92
  C:0F38H         LINE#         99
  C:0F3AH         LINE#         100
  C:0F3BH         LINE#         101
  C:0F3CH         LINE#         102
  C:0F3EH         LINE#         151
  C:0F41H         LINE#         155
BL51 BANKED LINKER/LOCATER V5.03                                                      07/03/2006  11:00:03  PAGE 3


  -------         ENDMOD        ?C_STARTUP

  -------         MODULE        SHTXX_DUMMY_CODE
  C:0000H         SYMBOL        _ICE_DUMMY_
  C:0D30H         PUBLIC        _calc_sht10
  C:0DEFH         PUBLIC        main
  D:0098H         PUBLIC        SCON
  D:0089H         PUBLIC        TMOD
  D:0088H         PUBLIC        TCON
  D:008DH         PUBLIC        TH1
  C:0F2BH         PUBLIC        init_uart
  -------         PROC          INIT_UART
  C:0F2BH         LINE#         27
  C:0F2BH         LINE#         30
  C:0F2EH         LINE#         31
  C:0F31H         LINE#         32
  C:0F34H         LINE#         33
  C:0F37H         LINE#         34
  -------         ENDPROC       INIT_UART
  -------         PROC          L?0017
  -------         ENDPROC       L?0017
  -------         PROC          _CALC_SHT10
  D:0028H         SYMBOL        p_humidity
  D:002BH         SYMBOL        p_temperature
  -------         DO            
  D:002EH         SYMBOL        rh
  D:0006H         SYMBOL        t
  D:0030H         SYMBOL        t_C
  D:0032H         SYMBOL        rh_lin
  -------         ENDDO         
  C:0D30H         LINE#         38
  C:0D36H         LINE#         45
  C:0D36H         LINE#         46
  C:0D3EH         LINE#         47
  C:0D49H         LINE#         53
  C:0D52H         LINE#         58
  C:0D5DH         LINE#         59
  C:0D5DH         LINE#         60
  C:0D76H         LINE#         61
  C:0D94H         LINE#         62
  C:0D96H         LINE#         64
  C:0D96H         LINE#         66
  C:0DC2H         LINE#         67
  C:0DD3H         LINE#         68
  C:0DD3H         LINE#         72
  C:0DE1H         LINE#         73
  -------         ENDPROC       _CALC_SHT10
  -------         PROC          MAIN
  -------         DO            
  D:0022H         SYMBOL        humi_val
  D:0024H         SYMBOL        temp_val
  D:0026H         SYMBOL        raw_data
  -------         ENDDO         
  C:0DEFH         LINE#         78
  C:0DEFH         LINE#         89
  C:0DEFH         LINE#         93
  C:0DF2H         LINE#         96
BL51 BANKED LINKER/LOCATER V5.03                                                      07/03/2006  11:00:03  PAGE 4


  C:0E03H         LINE#         97
  C:0E03H         LINE#         98
  C:0E09H         LINE#         99
  C:0E0CH         LINE#         100
  C:0E39H         LINE#         101
  C:0E46H         LINE#         103
  C:0E4FH         LINE#         106
  C:0E5BH         LINE#         107
  C:0E5BH         LINE#         108
  C:0E61H         LINE#         109
  C:0E64H         LINE#         110
  C:0EA1H         LINE#         111
  C:0EAFH         LINE#         113
  -------         ENDPROC       MAIN
  -------         ENDMOD        SHTXX_DUMMY_CODE

  -------         MODULE        ?C?UIDIV
  C:0B5CH         PUBLIC        ?C?UIDIV
  -------         ENDMOD        ?C?UIDIV

  -------         MODULE        ?C?SIDIV
  C:0BB1H         PUBLIC        ?C?SIDIV
  -------         ENDMOD        ?C?SIDIV

  -------         MODULE        ?C?ILDPTR
  C:0BE7H         PUBLIC        ?C?ILDPTR
  -------         ENDMOD        ?C?ILDPTR

  -------         MODULE        ?C?ISTPTR
  C:0C12H         PUBLIC        ?C?ISTPTR
  -------         ENDMOD        ?C?ISTPTR

  -------         MODULE        ?C?LMUL
  C:0C31H         PUBLIC        ?C?LMUL
  -------         ENDMOD        ?C?LMUL

  -------         MODULE        ?C?ULSHR
  C:0C80H         PUBLIC        ?C?ULSHR
  -------         ENDMOD        ?C?ULSHR

  -------         MODULE        PRINTF
  D:0028H         PUBLIC        ?_PRINTF517?BYTE
  D:0028H         PUBLIC        ?_PRINTF?BYTE
  D:0028H         PUBLIC        ?_SPRINTF517?BYTE
  D:0028H         PUBLIC        ?_SPRINTF?BYTE
  C:0862H         PUBLIC        _PRINTF
  C:0862H         PUBLIC        _PRINTF517
  C:085CH         PUBLIC        _SPRINTF
  C:085CH         PUBLIC        _SPRINTF517
  -------         ENDMOD        PRINTF

  -------         MODULE        ABS
  C:0F19H         PUBLIC        _abs
  -------         ENDMOD        ABS

  -------         MODULE        ?C?CLDPTR
  C:0C93H         PUBLIC        ?C?CLDPTR
BL51 BANKED LINKER/LOCATER V5.03                                                      07/03/2006  11:00:03  PAGE 5


  -------         ENDMOD        ?C?CLDPTR

  -------         MODULE        ?C?CLDOPTR
  C:0CACH         PUBLIC        ?C?CLDOPTR
  -------         ENDMOD        ?C?CLDOPTR

  -------         MODULE        ?C?CSTPTR
  C:0CD9H         PUBLIC        ?C?CSTPTR
  -------         ENDMOD        ?C?CSTPTR

  -------         MODULE        ?C?PLDIIDATA
  C:0CEBH         PUBLIC        ?C?PLDIIDATA
  -------         ENDMOD        ?C?PLDIIDATA

  -------         MODULE        ?C?CCASE
  C:0CFBH         PUBLIC        ?C?CCASE
  -------         ENDMOD        ?C?CCASE

  -------         MODULE        PUTCHAR
  C:0EF2H         PUBLIC        _PUTCHAR
  -------         ENDMOD        PUTCHAR

******************************************************************************
* RESTRICTED VERSION WITH 0800H BYTE CODE SIZE LIMIT; USED: 01F5H BYTE (24%) *
******************************************************************************

Program Size: data=36.1 xdata=0 code=1863
LINK/LOCATE RUN COMPLETE.  0 WARNING(S),  0 ERROR(S)
